:100000000207A60100010101010000C8EEC8740149
:10001000082275D88043878075BA03228F9930995A
:0A002000FDC29922905007EFF02274
:10002B000216E9EF14601014601624027027ED60BD
:10003B0003D28C22C28C22ED6003D28E22C28E227E
:10004B00ED600FE5C85403700CE5C854FC4401F592
:10005B00C82253C8FC22AF2511247BFF22D2BD221C
:10006B000212DBE539242DF8E6053922782A300710
:10007B0002782DE475F0011206CC0203CA2000EBC6
:10008B007F2ED2008018EF540F2490D43440D4FF2D
:10009B0030040BEF24BFB41A0050032461FFE53A80
:1000AB006002153A053DE53D7002053C30070D78C1
:1000BB002AE475F0011206CCEF02041002001C7446
:1000CB0003D2078003E4C207F5398B2A8A2B892CCC
:1000DB00E4F53AF53CF53DE53A60077F201200A9BF
:1000EB0080F5753BFFC201C200C202C203C205C24A
:1000FB0006C208120077FF700D3007057F00120053
:10010B00BAAF3DAE3C22B4255FC2D5C20412007714
:10011B00FF24D0B40A00501A75F00A783A30D5058E
:10012B0008B6FF0106C6A426F620D5047002D2033A
:10013B0080D924CFB41A00EF5004C2E5D2040202D6
:10014B00BAD20180C6D20080C0D20280BCD2D58088
:10015B00BAD20580B47F201200A92002077401B522
:10016B003A0040F112006EFF1200A90200E2D20821
:10017B00D206809512006EFB12006EFA12006EF919
:10018B004A4B7006798B7A037BFF20022EE53A608F
:10019B002A7E008E827583001203E360060EEE65E5
:1001AB003B70F0C2D5EBC0E0EAC0E0E9C0E0EE1274
:1001BB000301D0E0F9D0E0FAD0E0FB1203CAFF60F4
:1001CB00AAEBC0E0EAC0E0E9C0E01200A9D0E0244D
:1001DB0001F9D0E03400FAD0E0FBE53B0460DCD55C
:1001EB003BD980877BFF7A0279FDD202809C791004
:1001FB0080027908C206C2088008D2D5790A800429
:10020B00790AC2D5E53B047002F53BE4FAFDFEFF2B
:10021B0012006EFC7B0820011312006EFD7B103068
:10022B00000A12006EFE12006EFF7B20EC3382D5AB
:10023B0092D55013C3E43000069FFFE49EFEE420EA
:10024B0001039DFDE49CFCE4CBF8C201EC700CCFE8
:10025B00CECDCCE824F8F870F38017C3EF33FFEE64
:10026B0033FEED33FDEC33FCEB33FB994002FB0F1C
:10027B00D8E9EB300105F8D0E0C448B201C0E00A80
:10028B00EC4D4E4F78207B0070C2EAB53B0040BC72
:10029B00C0E0120303D0F0D0E0200104C4C0E0C4DE
:1002AB00B201C0F0120092D0F0D5F0EB0200E212D6
:1002BB0006DC017F5301F95801504C014C4201FD02
:1002CB004F020544020549016543020B5501EF46F8
:1002DB0001EF4501EF4703AB5001542D01582E019F
:1002EB007B2B015C2301792003942A011448000025
:1002FB0001733F3F3F00790AA2D520031430050953
:10030B00B910020404B9080104A2D5200602500159
:10031B00042002689202B53A005034C0E07F2030CE
:10032B0003197F30A20272067205500F12035AC2D4
:10033B0002C206C205C2087F30800F300503E9C038
:10034B00E01200A9300503D0E0F9D0E0B53ACC308B
:10035B0005177F30B9100C1200A97F583004077FA6
:10036B00788003B908031200A93002057F2D020023
:10037B00A97F202008F87F2B2006F322920280CF42
:10038B00286E756C6C2900D20112006E3001F8C218
:10039B0001783A30D50108F60201142D5043495823
:1003AB0012006E2403B405004001E49003A69312DF
:1003BB00009A743A12009AD203753A040201F9BBFF
:1003CB00010689828A83E0225002E722BBFE02E308
:1003DB002289828A83E49322BB010CE58229F58270
:1003EB00E5833AF583E0225006E92582F8E622BB45
:1003FB00FE06E92582F8E222E58229F582E5833AB9
:10040B00F583E49322BB010689828A83F022500292
:10041B00F722BBFE01F322EF8DF0A4A8F0CF8CF0F6
:10042B00A428CE8DF0A42EFE22BC000BBE0029EF1B
:10043B008DF084FFADF022E4CCF875F008EF2FFFC0
:10044B00EE33FEEC33FCEE9DEC984005FCEE9DFE8E
:10045B000FD5F0E9E4CEFD22EDF8F5F0EE8420D2D5
:10046B001CFEADF075F008EF2FFFED33FD40079844
:10047B005006D5F0F222C398FD0FD5F0EA22C2D573
:10048B00EC30E709B2D5E4C39DFDE49CFCEE30E70C
:10049B0015B2D5E4C39FFFE49EFE120434C3E49D62
:1004AB00FDE49CFC800312043430D507C3E49FFFAA
:1004BB00E49EFE22A3F8E0C5F025F0F0E58215825C
:1004CB0070021583E0C838F0E822BB010A89828AE2
:1004DB0083E0F5F0A3E022500687F009E71922BB71
:1004EB00FE07E3F5F009E3192289828A83E493F589
:1004FB00F074019322BB0110E58229F582E5833A62
:10050B00F583E0F5F0A3E0225009E92582F886F0A7
:10051B0008E622BBFE0AE92582F8E2F5F008E222A2
:10052B00E5832AF583E993F5F0A3E99322E88FF0AD
:10053B00A4CC8BF0A42CFCE98EF0A42CFC8AF0ED5F
:10054B00A42CFCEA8EF0A4CDA8F08BF0A42DCC3813
:10055B0025F0FDE98FF0A42CCD35F0FCEB8EF0A44B
:10056B00FEA9F0EB8FF0A4CFC5F02ECD39FEE43C05
:10057B00FCEAA42DCE35F0FDE43CFC2275F00875A9
:10058B008200EF2FFFEE33FECD33CDCC33CCC582C3
:10059B0033C5829BED9AEC99E58298400CF582EE7F
:1005AB009BFEED9AFDEC99FC0FD5F0D6E4CEFBE467
:1005BB00CDFAE4CCF9A88222B800C1B90059BA002F
:1005CB002DEC8BF084CFCECDFCE5F0CBF97818EF8A
:1005DB002FFFEE33FEED33FDEC33FCEB33FB10D78B
:1005EB0003994004EB99FB0FD8E5E4F9FA2278184C
:1005FB00EF2FFFEE33FEED33FDEC33FCC933C910A7
:10060B00D7059BE99A4007EC9BFCE99AF90FD8E0D8
:10061B00E4C9FAE4CCFB2275F010EF2FFFEE33FEAA
:10062B00ED33FDCC33CCC833C810D7079BEC9AE81D
:10063B0099400AED9BFDEC9AFCE899F80FD5F0DA9E
:10064B00E4CDFBE4CCFAE4C8F922EB9FF5F0EA9E8B
:10065B0042F0E99D42F0EC6480C864809845F0223A
:10066B00EB9FF5F0EA9E42F0E99D42F0E89C45F0E5
:10067B0022E8600FECC313FCED13FDEE13FEEF133A
:10068B00FFD8F122E493F8740193F9740293FA748E
:10069B000393FB22EC8EF0A4CCC5F0CCCDF8EFA4E9
:1006AB00CEC5F02DFDE43CFCE8A42EC8C5F03DFD05
:1006BB00E43CFCEFA4FFE5F028FEE43DFDE43CFC4C
:1006CB0022FAE6FB0808E6F925F0F618E6CA3AF630
:1006DB0022D083D082F8E4937012740193700DA32F
:1006EB00A393F8740193F5828883E473740293687F
:1006FB0060EFA3A3A380DF609700000972070002DD
:10070B00000101000102051022550F7103E800C81A
:10071B00555555555555555555555555555555557E
:10072B00555555555555555555555555555555556E
:10073B00555555555555555555555555555555555E
:10074B00555555555555555555555555555555554E
:10075B00000000000000000000000000000000008E
:10076B00000000000000000000000000000000007E
:10077B00000000000000000000000000000000006E
:10078B00000000000000000000000000000000005E
:10079B0000004200970000010D0000787FE4F6D8BE
:1007AB00FD75813E0207ED020BA7E493A3F8E493DA
:1007BB00A34003F68001F208DFF48029E493A3F849
:1007CB005407240CC8C333C4540F4420C8834004BB
:1007DB00F456800146F6DFE4800B0102040810207A
:1007EB004080900702E47E019360BCA3FF543F302E
:1007FB00E509541FFEE493A360010ECF54C025E01E
:10080B0060A840B8E493A3FAE493A3F8E493A3C8D5
:10081B00C582C8CAC583CAF0A3C8C582C8CAC58366
:10082B00CADFE9DEE780BEAC08AD09AE0AAF0B78D4
:10083B0010EC4D4E4F70047CA57DA5C3EC13FCED65
:10084B0013FDEE13FEEF13FF5010EC64CCFCED64C4
:10085B004CFDEE644EFEEF64CEFFD8DF8C088D09A5
:10086B008E0A8F0BEE547FFE228E088F0974A5F52E
:10087B000AF50B22524620547820546573742E0DC2
:10088B000A00547826527820646F6E652E0A005445
:10089B0078206661696C2E0A006D6F64653D5B257F
:1008AB0062755D0D0A0052465F456E746572527833
:1008BB004D6F64650D0A0072616E645F6E756D3D00
:1008CB005B2562755D0D0A0072665F63683D5B2593
:1008DB0062755D0D0A00EF540FFEEF54F0FCBC1077
:1008EB0005E4F52E800AEC64306002419D752EFB09
:1008FB00E52E5403FF240CF5F8ED5401D39400407E
:10090B000D12000B8002C333D8FC42F9800C12008D
:10091B000B8002C333D8FCF452F9EF240DF5F8ED3C
:10092B005402D39400400D12000B8002C333D8FC49
:10093B0042F9800C12000B8002C333D8FCF452F93D
:10094B00E52E5403240EF5F8ED5404D39400400D1A
:10095B0012000B8002C333D8FC42F9800C12000B3F
:10096B008002C333D8FCF452F9EB64037018F1B175
:10097B0012000B8002C333D8FCF4FD52F9EF04F5DF
:10098B00F8ED52F98048F1B1EB5401D39400400DCE
:10099B0012000B8002C333D8FC42F9800C12000BFF
:1009AB008002C333D8FCF452F9EF04F5F8EB540290
:1009BB00D39400400D12000B8002C333D8FC42F9D4
:1009CB00800C12000B8002C333D8FCF452F9AF2E0B
:1009DB00EFC4135401240AF5F8EB25E02404F58247
:1009EB00E43400F19F400D12000B8002C333D8FC9E
:1009FB0042F9800C12000B8002C333D8FCF452F97D
:100A0B00AF2EEFC454012404F5F8CFEBCFEF25E064
:100A1B002403F582E43400F19F400D12000B800299
:100A2B00C333D8FC42F9800C12000B8002C333D8BD
:100A3B00FCF452F9AF2EEFC4131354012406F5F84E
:100A4B00E52D5401D39400400D12000B8002C333EB
:100A5B00D8FC42F9800C12000B8002C333D8FCF493
:100A6B0052F9AF2EEFC413131354012408F5F8E514
:100A7B002D5402D39400400C12000B8002C333D8C8
:100A8B00FC42F922CFEECFF1C18002C333D8FCF484
:100A9B0052F922EF4D4BF598E52D14B40800507325
:100AAB00900AB975F003A4C58325F0C58373020AB8
:100ABB00D1020ADE020AE5020AEC020AF3020AFE7E
:100ACB00020B05020B0C75D88043878075BA027533
:100ADB00AA5F2212001275AA302212001275AA9870
:100AEB002212001275AACC22758920758DF7758B91
:100AFB00F7801712001275AAE62212001275AAF3DC
:100B0B0022758920758DFD758BFD43884075D84006
:100B1B0043878022CCEFCCEC7021C28CBD0209E55F
:100B2B002EF58C858C8A8008E52DF58CE52EF58AC3
:100B3B005389FBE58954FC4DF58922EC6401702641
:100B4B00C28EBD0209E52EF58D858D8B8008E52DB6
:100B5B00F58DE52EF58B5389BFEDC454F0FFE58978
:100B6B0054CF4FF58922EC6402703053C8FCE52D4D
:100B7B00FFF5CDAE2EE52EF5CC8FCB8ECAEBC43365
:100B8B0033335480FFE5C8547F4FF5C8ED7009E54A
:100B9B00C854E74410F5C82253C8E722E4F5227580
:100BAB0023FAF524752502F526F527F528F52912E4
:100BBB0011397FE87E0312127CD1F8F153B1B4F1F5
:100BCB0036752D01E4FBFD7F3211E1D2AF7BFF7A4D
:100BDB0008797F81BDE50C602524F0601524F06059
:100BEB000C24C070167BFF7A08798D800B7522015F
:100BFB0080097BFF7A08799A1200D0E4F50C121267
:100C0B009DEF601E7522017524010523E523C39416
:100C1B00094003E4F5237BFF7A0879A485232D1281
:100C2B0000D0E523B4090050AC900C3BF828287396
:100C3B00020C56020C79020C90020CA7020CC20299
:100C4B000CD6020CE3020CF3020D4DE5246006F109
:100C5B0073B1B2F131E522700261E0E4F522F11ECD
:100C6B00900008E0F12A600280177FA0A148E524DC
:100C7B006007F1737F28120024E522700261E0F116
:100C8B00257FB0A148E5246007F1737F5012002443
:100C9B00E522700261E0F1257FB0A148E5247002E6
:100CAB0061E0E4F5247F02120024F17A7BFF7A08DD
:100CBB0079B11200D061E0E524700261E0E4F52423
:100CCB00F522B1B2F13112171B61E0E5247002611C
:100CDB00E0E4F5247F28800BE524700261E0E4F565
:100CEB00247F5012002461E0E524600FE4F524B169
:100CFB00B2F136752201E4F528F529121AFD402BC5
:100D0B00E4F528F52911327C007D291204898D2602
:100D1B00E52625E0F525D3945040037525501200A8
:100D2B00617A0879C285252D1200D0E52270026107
:100D3B00E00529E52970020528F1257FB01215463B
:100D4B0061E0E524600CE4F524F525752201F52816
:100D5B00F529121AFD4022E4F528F529F52205257F
:100D6B000525E525D3945040037525021200617AC1
:100D7B000879D385252D1200D0E522700261E0E4BD
:100D8B00F5220529E52970020528F1287FB01215F7
:100D9B004661E0EF14600A14600A24027008D2A9BD
:100DAB0022D2AB22D2AD22F1427B017A0079008BA9
:100DBB002A8A2B892C7D017F007E01D1CE1211BA9C
:100DCB00E4FF121AE0D1F19000041203E3FF1218B2
:100DDB0024D1F19000031203E3FF121582D1F1121B
:100DEB0004D524A0FF120024D1F190000A1203E3D2
:100DFB00FF12172FD1F19000021203E3FF121754C9
:100E0B007F01121AB7121AF0C0E0EAC0E0E9C0E0A5
:100E1B00F1A7FDD0E0F9D0E0FAD0E0FB12194512B2
:100E2B001AF0C0E0EAC0E0E9C0E0F1A7F531D0E08C
:100E3B00F9D0E0FAD0E0FBE4FF12188F7D40E4FF1D
:100E4B0012198ED1F19000051203E3FF121866D12F
:100E5B00F1900013120500FFAEF01219F5D1F190CD
:100E6B0000051203E364017039900011120500FFB5
:100E7B00AEF0121A1A7D037FFA7E001219ABD1F174
:100E8B009000081203E3FF12199BD1F19000061298
:100E9B0003E3FF121AA7D1F19000071203E3FDE45D
:100EAB008014E4FD7FFAFE1219AB7F0112199BE44B
:100EBB00FF121AA7E4FDFFF1C87D017F38121ACD8E
:100ECB00020068CBEFCBEB600875FC0CED60128079
:100EDB000975FC0DED6007CFEECFEF42FD22CFEE93
:100EEB00CFEFF452FD22AB2AAA2BA92C227D017F36
:100EFB0002F14C7F01F14C7F087E00D1CEE4F52D41
:100F0B007B017D017F3111E1752D087B40E4FD7F75
:100F1B0040419E90506174E1F022E4F522F11E7C79
:100F2B00007D157B40227F02120024F18054FEF0DD
:100F3B009050607401F02275FC0143FD0153FDFEDE
:100F4B00227E00D1CE7D01227D017F107E00D1CE8D
:100F5B00752DFA752ECBE4FBFD7F02711F7F02B15D
:100F6B009E7D017F0202002EE4F52475220122F101
:100F7B0080440180BA905060E4F0F11EF190F1973B
:100F8B00905000E02290506174E2F02290500CE0FF
:100F9B0044F0F022F583E493D3940022AA2BA92CDE
:100FAB0090000B0203E3AF2EEF13135403FFF5F87E
:100FBB002290503CE0FEC8EFC874010822ED600C93
:100FCB00F1BC8002C333D8FC4EF0800BF1BC800225
:100FDB00C333D8FCF45EF090503CE0543F6006A362
:100FEB00E04404F02290503DE054FBF022E13B8DB5
:100FFB002B90000075FC03EF14603F14605C1470C1
:10100B000201C22403600201E7E52B601F11E8E532
:10101B00FB20E0FB75FC06E5FD30E70201E711F272
:10102B0070020583310250EF11F980EB53FDFD1176
:10103B00EBE5FB20E00201E780F7E52B600E43FDBB
:10104B000111EBE5FB20E00201E780F753FDFE11F8
:10105B00EBE5FB20E00201E780F7E52B6055E5FDB2
:10106B0020E279E5FD4404F52CE5FD30E72411E899
:10107B00E5FB20E0FB75FC06AFFDEF20E70E11F260
:10108B0070020583310250ED11F980E975FC0353B1
:10109B00FD3F311143FD1075FC08AFFDEF20E60E4F
:1010AB0011F270020583310250ED11F980E975FCE4
:1010BB0008800053FDFB22E52B601EE5FD20E31CA1
:1010CB0043FD0875FC0AE5FD20E51111F2700205E0
:1010DB0083310250F111F980ED53FDF72243FD02EC
:1010EB0075FA1643FB01220582E582AE8322C2AF5D
:1010FB0043F70143F7012214FFE4FCFD7BFA7AFF6F
:10110B00F9F8C302065575FC0843FD0C75FC085332
:10111B00FDEF75FC0343FD0475FC082275FC03EF22
:10112B00C4333354C0FFE5FD543F4FF5FD2231ABC3
:10113B006401701A75FC0DAEFD8E2AE52A20E006BF
:10114B0075FC0D43FD0131B275FC0D852AFDEFB425
:10115B00020675FC0443FD803190E4FF31277D01CD
:10116B007F02120FFA7D017F03120FFA9081D3E4F5
:10117B0093B401047F0231279081D3E493B402042A
:10118B007F033127227F557EAA7DAA7C559081CF84
:10119B0012068FC312066B60067D1A7F20516322E5
:1011AB009081D3E493FF22905036E04480F02212DA
:1011BB000F4231B290503CE4F09050087464F090C0
:1011CB00503374C4F090503B740BF090503D7498B6
:1011DB00F0905006E4F090503E74B2F0905058747A
:1011EB0030F0A374F0F090505C7405F090505E7486
:1011FB0080F09050857440F0905087740AF0A3747F
:10120B004AF0A37402F09050037419F0A374ECF03D
:10121B00A37487F090501E7403F090500B745BF026
:10122B009050347401F0905041E4F0A37444F0906A
:10123B005054744AF0A37440F0A37422F090507A87
:10124B00743AF0A374FFF0A3747BF0905000740415
:10125B00F09050617473F0228F2B8D2C75FC06E58A
:10126B00FD548F4FF5FD75FC10ED25E04480F5FD29
:10127B0022E4FDFCC3ED9FEC9E5016E4FBFA000B41
:10128B00BB00010ABA03F7BBE8F40DBD00010C80EB
:10129B00E32230B20479018002E4F9E9700DE50D27
:1012AB00702351D3701F750D01801AE96017E50D7E
:1012BB00B4011251D3600EE50DB40106E4F50D7FB8
:1012CB000122E4F50D7F00227F2C7E01517CE92267
:1012DB00C0E0C0F0C083C082C085C084C09253926E
:1012EB00FEC0D0E8C0E0E9C0E0EAC0E0EBC0E0EC53
:1012FB00C0E0EDC0E0EEC0E0EFC0E0D1C88F0CE580
:10130B000C24A07013900006E0600D7E007F557DCD
:10131B00407152900096EFF0120F90120F97D0E0A1
:10132B00FFD0E0FED0E0FDD0E0FCD0E0FBD0E0FA57
:10133B00D0E0F9D0E0F8D0D0D092D084D085D08254
:10134B00D083D0F0D0E032CBEFCBCAEECA90506353
:10135B00E0FFC9EFC9F53E9081E3E49320E402710D
:10136B0099E53ED39D50219050617461F0AF3E15CD
:10137B003EEF6010905062E08B828A83F00BBB00D3
:10138B00010A80E9B17B8002E4F9CFE9CF227FDC4F
:10139B007E05EF4E600BEF1FCCEECC70011E4C7038
:1013AB00F5228F2F905080D1D04480CFEFF0E52FD6
:1013BB004460905075F0905072E04410F0E4F530BA
:1013CB00E52F25E025E08530F0A4252FFF12002422
:1013DB0090503EE0F5315331F8433104E531F09054
:1013EB00507FE04480F09050A2E030E5F990507FC0
:1013FB00E044409164E054BFF07F407E06719D90C5
:10140B0050A5E030E5F97F0A7E00719D90507FE09A
:10141B00547FF09050A5E0541FFFE530FDC3746D71
:10142B009DFD745094008D82F583EFF00530E5300F
:10143B00C39404408B905072E054EFF090503EE018
:10144B00FFCF54F8CFCF4402CFEFF090506A915CAE
:10145B00A3E014F0A3E014F022F07F057E00619D61
:10146B008F2F8D30E4F531B1157C037D1612069F5D
:10147B00780712067C91F4453191E491D6E0547FC4
:10148B00F091D691DC40E0E4F531B115E4FCFD7B45
:10149B009C7AC6790DF81205387B007AF4790178BD
:1014AB00001205C391F4FFE5312405FEEF4E91E4E4
:1014BB009165E0547F916491DC40CFE52FC454F0EB
:1014CB00FFE530540F4F90506FF0227F847E036105
:1014DB009D0531E531C3940522F090507DE533F045
:1014EB00E532A3F0E04480F0228E348F35E53524CD
:1014FB0005FFE43534FE7C007D0A1204348E328FF6
:10150B0033905072E054F0F0E022E530FB75F004BC
:10151B00A42401FFE435F0FEAD317C00120422CC93
:10152B00EECCCDEFCDEB25E0FFE433FEED2FFFEC62
:10153B003EFEEF2462FFEE3409FE22C9EFC9E4FA46
:10154B008C2A8D2B9081E39320E4027199EBD39439
:10155B0040501C905061E9F0EAC39B5010CFEACF8A
:10156B000AE52B2FF582E4352AD1D880EBB17B220B
:10157B0090506174FFF0228F2D905007E0F52E9064
:10158B005009E054FCF0905033E054CFF09050767B
:10159B00E054E0F090507FE054C0F0E52D702090C7
:1015AB005009E0F0905033E0F09050247424F09008
:1015BB005076E04418F090507FE04419F08058E5E5
:1015CB002D64017024905009E04401F0905033E0F9
:1015DB004410F090502474A4F0905076E0441FF027
:1015EB0090507FE04432F0802EE52D6402702890FD
:1015FB0050437487F0905009E04403F0905033E06F
:10160B004430F09050247404F0905076E04412F083
:10161B0090507FE0441DF0120FF87D077F05D13A03
:10162B007F0A71ADAF2DD16E905007E52EF0229150
:10163B006B90503BE04402F0905070E04408F09007
:10164B0050A2E030E5F990505EE04408F09050A2D3
:10165B00E030E4F990505EE054F7F0905070E054B5
:10166B00F7F022905000E0FE120F3B905000E04448
:10167B0001F090500BE054BFF090504BE04480F0E1
:10168B0090505FBF02057462F080037460F090505D
:10169B0005E04410F0905037E04408F09050ABE078
:1016AB004401F09050AAE030E7F9905005E054EF78
:1016BB00F0905037E054F7F0D1E0EEF02290500C60
:1016CB00E054F0FF22E0FFCF543FCFCF22F583E071
:1016DB00905062F022905060E4F090500022C0E0F5
:1016EB00C083C082C085C084C0925392FEC2C69094
:1016FB000098E004F07006900097E004F0D092D0D0
:10170B0084D085D082D083D0E032905060E4F02238
:10171B0090503BE054FDF0E04402F0F11590503551
:10172B0074AEF022E4FE905000E054F9F0EF146038
:10173B000B14600C2402700AE4FE80067E02800209
:10174B007E06905000E04EF02290500AE05480F05C
:10175B00A3E054C7F0EFB40E004003021809901732
:10176B0070F828287302179A0217A10217A80217FC
:10177B00AF0217B60217BD0217C40217CB0217D25E
:10178B000217D90217E00217EC0217F30217FF1228
:10179B001AE644078044121AE64409803D121AE601
:1017AB00440B8036121AE6440E802F121AE64415AB
:1017BB00802812180A440E802112180A4411801A2C
:1017CB0012180A4414801312180A4417800C1218AA
:1017DB000A441D800512180A4426F0A3E04408F0C1
:1017EB002212180A4426800512180A4438F0A3E086
:1017FB004418F022110A447FF0A3E04438F0229001
:10180B005009E054FBF0A3E022EF9050356005E067
:10181B004401F022E054FEF022E4FE90503D749817
:10182B00F0EF60131460181470267E40905001E4A2
:10183B00F0905006F08002E4FE7F01111480117EBF
:10184B0080E4FF111490503DE04460F0E054E7F069
:10185B00905000E0543FF0E04EF022EF70059050B6
:10186B0001F022BF0107905001E04401F02290509B
:10187B0002E0543FF0E0FEEF24FEC4333354C0FFCC
:10188B00EE4FF0228B2E8A2F8930CCEFCCE4F53241
:10189B00AF311179CFECCF7D013123CFCFEF146076
:1018AB002114602F14603314603714603B240570CF
:1018BB003D753350753410E532C3953150303103DB
:1018CB0080F5753350753415E532C39531501F31A2
:1018DB000380F511FA90501BF02211FA90501AF078
:1018EB002211FA90501DF02211FA90501CF022ABED
:1018FB002EAA2FA9300203CAAB2EAA2FA9308532EC
:10190B00827583001203E3FFE5342532F582E4355B
:10191B0033F583EFF0053222ED600F905002120F7A
:10192B00BF8002C333D8FC4EF022905002120FBF7F
:10193B008002C333D8FCF45EF0228B2D8A2E892FC4
:10194B009000997401F0A37450F0A37426F0CFEDBE
:10195B00CF1179CFEDCF1DEF6028AB2D052FE52FE4
:10196B00AA2E7002052E14F91203CAFF900099E0FB
:10197B00FBA3E475F0011204BFA9F0FAEF120410F7
:10198B0080D122742B2FF582E43450F583EDF022B5
:10199B00EF90503D6005E04401F022E054FEF02250
:1019AB00CBEDCBC3EF94FAEE9400402DD3EF94A084
:1019BB00EE940F50247C007DFA1204348F2DE52D0C
:1019CB00D394004002152D905006E0540FF0E0FF29
:1019DB00E52DC454F0FEEF4EF0EBD3940F500A906C
:1019EB005006E054F0F0E04BF022EE510E905042D6
:1019FB00E054C0F0E0CCEFCC4CF0A3E054C0F0E0EE
:101A0B004FF022C4F854F0C8EFC4540F48FF229093
:101A1B005033E0C45403FD905040E054C0F0BD017E
:101A2B001FD3EF9400EE940440047E047F0090508B
:101A3B0040E0FDEF24F0FFEE34FF510EED4FF022AE
:101A4B00ED702AD3EF9400EE940840047E087F00DB
:101A5B00905040C083C082E0FDEF24E0FFEE34FFE6
:101A6B00FE7805EFCEC313CE13D8F98028D3EF94AD
:101A7B0000EE942040047E207F00905040C083C035
:101A8B0082E0FDEF2480FFEE34FFFE7807EFCEC33C
:101A9B0013CE13D8F94DD082D083F022EF90503D66
:101AAB006005E04402F022E054FDF022EF70089054
:101ABB00503DE054E7F022BF010790503DE0441841
:101ACB00F022ED9050007004E04FF022E0FEEFF4B6
:101ADB00FFEE5FF02275FC178FFD22905009E0445A
:101AEB0004F0A3E022AB2AE52C240CF9E4352BFA05
:0E1AFB00EB22C3E529942CE528648094812217
:00000001FF
